:1000000000308A0049290000FF00030E8301A1008F
:100010007F08A0000A08A8008A01A00E0408A20018
:100020007708A3007808A4007908A5007A08A6003C
:100030007B08A700831383128B1E20280B193328FB
:10004000220884002308F7002408F8002508F90096
:100050002608FA002708FB0028088A00210E8300E2
:10006000FF0E7F0E09008A11352829080139013C4D
:1000700003193C2800303D280130F8007818422848
:100080003B1043283B14831685178312851B4A288F
:100090003B185128831685178312851F56283B1855
:1000A00056282B0F54285528AB0A5728AB01831626
:1000B00005168312051A5E283B1865288316051657
:1000C0008312051E6A283B186A282A0F68286928A7
:1000D000AA0A6B28AA01831686158312861972282C
:1000E0003B187928831686158312861D7E283B18B7
:1000F0007E282C0F7C287D28AC0A7F28AC01831633
:1001000005178312051B86283B188D2883160517B3
:100110008312051F92283B1892282D0F90289128B2
:10012000AD0A9328AD01A90A29080139013C031938
:100130009B2800309C280130F8007818A1283B103B
:10014000A2283B1483161C1BA9288312AF14AB28CA
:1001500083168312AF1083169C1BB22883122F14B0
:10016000B428831683122F103B1CB9281B3095002E
:10017000BB2837309500073083169C0005080630F1
:10018000F700F70BC12800001C0883120D1383161B
:10019000851483128518D1282E0FCF28D028AE0AB7
:1001A000D228AE010A3083169C0005080C38850061
:1001B0000630F700F70BDA2800001C0883120D1335
:1001C0002E08033C0318F7282F19F72883168613E7
:1001D000831286138316061383120617831686125C
:1001E000831286128316061283120616F6280B1146
:1001F0008A1120280830BA02031C09293A308400E9
:100200000310800C00080319092907290000800B3E
:10021000062900340B138B138B1B0B293708B900ED
:100220003608B800B808031D1829B908031933297E
:100230008316861083128614831606118312061104
:100240003408BA00FA2083160611831206158316A5
:100250008610831286103408BA00FA203808031971
:10026000B903B8031229C0308B0400343530840040
:100270000008031948290230F800F701F70B3E295E
:10028000F80B3D299730F700F70B4429800B3B29E9
:10029000003484011F308305703083168F001F12D5
:1002A0009F121B0880399B0007309C008312A90114
:1002B000AA01AB01AC01AD01AE012F10AF102F119F
:1002C000831606138312061383168613831286136E
:1002D0008316061283120612831686128312861262
:1002E000723083168F001F129F121B0880399B00EB
:1002F00083121F1094128316061186140612003002
:1003000083129400831694000108C03901388100DB
:10031000831290010030F8000438920036308316C2
:1003200092000610831206100C3097001B309500C7
:100330000A3083169C0005080C3885000630F7004B
:10034000F70BA02900001C0883120D130730831639
:100350009C0005080630F700F70BAC2900001C08CC
:1003600083120D138F3083169D0003308312B50066
:10037000E830B400B701C830B6000A213230B50009
:1003800036210330B500E830B400B701C830B600FC
:100390000A21073083169C0005080630F700F70B8A
:1003A000CF2900001C0883120D13831685148312B5
:1003B00085189C2B0A3083169C0005080C38850094
:1003C0000630F700F70BE22900001C0883120D131A
:1003D0002F158B16C0308B042E08643C0318F829A7
:1003E0000330B5002030B400B7016430B6000A21F4
:1003F0003230B50036212F1C102A0330B500E8300A
:10040000B400B701C830B6000A210A30B500362161
:100410000330B500E830B400B701C830B6000A2197
:100420003230B5003621AF1C2A2A0730B500D03053
:10043000B4000130B7002C30B6000A210A30B500F4
:1004400036210730B500D030B4000130B7002C3071
:10045000B6000A213230B50036212B080A3C0318B9
:100460003A2A0B30B500B830B4000130B7009030F4
:10047000B6000A213230B50036212D080A3C031897
:100480004A2A0F30B500A030B4000130B700F43074
:10049000B6000A213230B50036212A080A3C03187A
:1004A0005A2A1330B5008830B4000130B700F43058
:1004B000B6000A213230B50036212C080A3C031858
:1004C0006A2A1730B5007030B4000230B7005830D7
:1004D000B6000A213230B50036212E08643C0318DC
:1004E000752A2F1C752AAF18762AEC290130B30023
:1004F000F430B2003308033C031C922A031D842A03
:1005000032081F3C031C922A3308B5003208B4009D
:100510003308B7003208B6000A216430B207031866
:10052000B30A7A2A0430B400FA30B5003621B40B8D
:10053000942A8316061383120613831686138312D6
:1005400086138316061283120612831686128312EE
:10055000861283168612831286128316061283125F
:1005600006160430B400FA30B5003621B40BB32AB5
:1005700083160612831206128316861283128612BF
:100580000430B400FA30B5003621B40BC22A831609
:100590000612831206128316861283128616043000
:1005A000B400FA30B5003621B40BD12A83160612F6
:1005B0008312061283168612831286120430B40048
:1005C000FA30B5003621B40BE02A0330B5007030A4
:1005D000B400B7016430B6000A210430B400FA3028
:1005E000B5003621B40BEF2A8316861383128613C7
:1005F00083160613831206170430B400FA30B500D0
:100600003621B40BFE2A83160613831206138316B3
:100610008613831286130430B400FA30B5003621F5
:10062000B40B0D2B83160613831206138316861341
:10063000831286170430B400FA30B5003621B40BAB
:100640001C2B83160613831206138316861383123C
:1006500086130430B400FA30B5003621B40B2B2BCE
:100660000330B5007030B400B7016430B6000A2121
:100670000430B400FA30B5003621B40B3A2B83169F
:1006800086138312861383160613831206178316A6
:1006900086128312861283160612831206160430FF
:1006A000B400FA30B5003621B40B512B8316061373
:1006B000831206138316861383128613831606127B
:1006C0008312061283168612831286120430B40037
:1006D000FA30B5003621B40B682B8316061383124B
:1006E0000613831686138312861783160612831247
:1006F000061283168612831286160430B400FA306E
:10070000B5003621B40B7F2B831606138312061314
:10071000831686138312861383160612831206121B
:1007200083168612831286120430B400FA30B500A4
:100730003621B40B962B762A8B16C0308B04B10170
:100740000130B000B108031DBC2B3008053C031C70
:10075000BC2B0530B2008630B5003621B20BAB2B76
:100760000330B500E830B400B701C830B6000A2144
:10077000B00A0319B10AA22B0108963C031CC92B2D
:1007800083168613831286138316061383120617A5
:10079000D12B831606138312061383168613831236
:1007A00086130108963C031CDE2B831686128312E7
:1007B00086128316061283120616E62B831606127D
:1007C000831206128316861283128612AF1C522CD5
:1007D0008316061383120613831686138312861755
:1007E0008316061283120612831686128312861649
:1007F000B430B50036218316061383120613831610
:10080000861383128613831606128312061283162A
:10081000861283128616B101B0013108133C031C05
:100820002F2C031D172C3008873C031C2F2CAF1CCA
:100830001B2C2F1C2B2C83160613831206138316D6
:1008400086138312861783160612831206128316E6
:10085000861283128616B00A0319B10A0D2C83166C
:1008600086138312861383160613831206178316C4
:1008700006128312061283168612831286166430BD
:10088000B5003621831606138312061383168613CA
:10089000831286138316061283120612831686129B
:1008A000831286122F1CBE2C831606138312061386
:1008B0008316861383128617831606128312061276
:1008C0008316861283128616B430B500362183163D
:1008D0000613831206138316861383128617831654
:1008E0000612831206128316861283128612B10133
:1008F000B0013108133C031C9B2C031D832C3008D2
:10090000873C031C9B2C2F1C872CAF1C972C831619
:100910000613831206138316861383128617831613
:100920000612831206128316861283128616B00AE6
:100930000319B10A792C8316061383120613831642
:1009400086138312861783168612831286128316E5
:100950000612831206166430B5003621831606137C
:1009600083120613831686138312861383160612C8
:100970008312061283168612831286122B080A3CF3
:1009800003186E2D8316861383128613831606139F
:100990008312061783168612831286128316061296
:1009A00083120616B101B0013108133C031CFA2C66
:1009B000031DDE2C3008873C031CFA2C2F18E22C78
:1009C000AF1CF62C831606138312061383168613A8
:1009D0008312861783160612831206128316861256
:1009E000831286166430B5003621BC2BB00A031979
:1009F000B10AD42C8316861383128613831606132A
:100A000083120617831606128312061283168612A5
:100A100083128616B101B0013108273C031C6E2DEC
:100A2000031D162D30080F3C031C6E2D2F181A2D98
:100A3000AF1C2E2D831606138312061383168613FE
:100A400083128617831606128312061283168612E5
:100A5000831286166430B5003621BC2B2D08053C68
:100A60000318422D831686138312861383160613EA
:100A700083120617831686128312861283160612B5
:100A8000831206162A08053C0318562D83160613F2
:100A90008312061383168613831286178316861213
:100AA0008312861283160612831206162B08053C43
:100AB00003186A2D83168613831286138316061372
:100AC00083120617831606128312061283168612E5
:100AD00083128616B00A0319B10A0C2D2A080A3CA3
:100AE00003181E2E8316861383128613831606138D
:100AF0008312061783168612831286128316061235
:100B000083120616B101B0013108133C031CAA2D53
:100B1000031D8E2D3008873C031CAA2D2F18922D03
:100B2000AF1CA62D83160613831206138316861395
:100B300083128617831606128312061283168612F4
:100B4000831286166430B5003621BC2BB00A031917
:100B5000B10A842D83160613831206138316861397
:100B60008312861783168612831286128316061244
:100B700083120616B101B0013108273C031C1E2E5A
:100B8000031DC62D30080F3C031C1E2E2F18CA2D26
:100B9000AF1CDE2D831606138312061383168613ED
:100BA0008312861783160612831206128316861284
:100BB000831286166430B5003621BC2B2D08053C07
:100BC0000318F22D831686138312861383160613D9
:100BD0008312061783168612831286128316061254
:100BE000831206162A08053C0318062E83160613E0
:100BF00083120613831686138312861783168612B2
:100C00008312861283160612831206162B08053CE1
:100C100003181A2E8316861383128613831606135F
:100C20008312061783160612831206128316861283
:100C300083128616B00A0319B10ABC2D2D080A3C8E
:100C40000318582E83160613831206138316861371
:100C50008312861783168612831286128316061253
:100C6000831206166E30B500362183168613831262
:100C70008613831606138312061783160612831231
:100C8000061283168612831286163230B50036217C
:100C90008316061383120613831686138312861394
:100CA0008316061283120612831686128312861288
:100CB0002C080A3C0318922E83160613831206137F
:100CC0008316861383128617831686128312861262
:100CD00083160612831206166E30B500362183166F
:100CE0008613831286138316061383120617831640
:100CF000061283120612831686128312861632306B
:100D0000B500362183160613831206138316861345
:100D10008312861383160612831206128316861216
:080D200083128612BC2B630054
:04400E00383FFC3FFC
:00000001FF
